:10000000020A03750940E4F50E750DE1F50CF50BD8
:10001000751001FB7A0079097F021207FF7D017FCD
:10002000011209A553BAFE227DA37C08ED1D7001C3
:0F0030001C144C70F7EF1F70011E144E70EA2263
:10004300020954E518240CF8E6051822780930074C
:1000530002780CE475F0011207C90206192000EBBF
:100063007F2ED2008018EF540F2490D43440D4FF55
:1000730030040BEF24BFB41A0050032461FFE519C9
:1000830060021519051CE51C7002051B30070D786D
:1000930009E475F0011207C9EF020781020A197416
:1000A30003D2078003E4C207F5188B098A0A890B78
:1000B300E4F519F51BF51CE51960077F2012008193
:1000C30080F5751AFFC201C200C202C203C205C293
:1000D30006C20812004FFF700D3007057F001200A3
:1000E30092AF1CAE1B22B4255FC2D5C20412004FCF
:1000F300FF24D0B40A00501A75F00A781930D505D8
:1001030008B6FF0106C6A426F620D5047002D20362
:1001130080D924CFB41A00EF5004C2E5D2040202FE
:1001230092D20180C6D20080C0D20280BCD2D580D8
:10013300BAD20580B47F201200812002077401B572
:10014300190040F1120046FF1200810200BAD208E2
:10015300D2068095120046FB120046FA120046F9B9
:100163004A4B700679637A037BFF20022EE5196000
:100173002A7E008E8275830012063260060EEE65BB
:100183001A70F0C2D5EBC0E0EAC0E0E9C0E0EE12BD
:1001930002D9D0E0F9D0E0FAD0E0FB120619FF60F3
:1001A300AAEBC0E0EAC0E0E9C0E0120081D0E0249D
:1001B30001F9D0E03400FAD0E0FBE51A0460DCD5A5
:1001C3001AD980877BFF7A0279D5D202809C791075
:1001D30080027908C206C2088008D2D5790A800451
:1001E300790AC2D5E51A047002F51AE4FAFDFEFF96
:1001F300120046FC7B08200113120046FD7B1030E1
:10020300000A120046FE120046FF7B20EC3382D523
:1002130092D55013C3E43000069FFFE49EFEE42012
:1002230001039DFDE49CFCE4CBF8C201EC700CCF10
:10023300CECDCCE824F8F870F38017C3EF33FFEE8C
:1002430033FEED33FDEC33FCEB33FB994002FB0F44
:10025300D8E9EB300105F8D0E0C448B201C0E00AA8
:10026300EC4D4E4F78207B0070C2EAB51A0040BCBB
:10027300C0E01202DBD0F0D0E0200104C4C0E0C42F
:10028300B201C0F012006AD0F0D5F0EB0200BA124E
:1002930007D901575301D15801284C01244201D5F4
:1002A3004F01DD4401DD49013D4301E35501C746EB
:1002B30001C74501C747038350012C2D01302E018F
:1002C300532B013423015120036C2A00EC48000016
:1002D300014B3F3F3F00790AA2D5200314300509A3
:1002E300B910020404B9080104A2D5200602500182
:1002F300042002689202B519005034C0E07F203018
:1003030003197F30A20272067205500F120332C224
:1003130002C206C205C2087F30800F300503E9C060
:10032300E0120081300503D0E0F9D0E0B519CC30FC
:1003330005177F30B9100C1200817F583004077FF6
:10034300788003B908031200813002057F2D020073
:10035300817F202008F87F2B2006F322920280CF92
:10036300286E756C6C2900D2011200463001F8C268
:1003730001781930D50108F60200EC2D5043495895
:100383001200462403B405004001E490037E931257
:100393000072743A120072D2037519040201D1EF8C
:1003A300D394077480948040037FFF22120619FEC2
:1003B300D394037480948040037FFF22EF7044EE54
:1003C300700B900001120632F452935294120619E4
:1003D3006401700B9000011206324293F45294129E
:1003E3000619FE6402700A9000011206324293421B
:1003F30094EE6403700D900001120632FEF45293E2
:10040300EE4294EF64017046120619FE700B9000E1
:1004130001120632F452915292EE6401700B900075
:10042300011206324291F452921206196402700AC2
:10043300900001120632429142921206196403702F
:100443000D900001120632FEF45291EE4292EF64D7
:10045300027046120619FE700B900001120632F468
:1004630052955296EE6401700B90000112063242CF
:1004730095F452961206196402700A90000112064E
:1004830032429542961206196403700D90000112D0
:100493000632FEF45295EE4296EF6403704612065E
:1004A30019FE700B900001120632F452B152B2EEF3
:1004B3006401700B90000112063242B1F452B21281
:1004C30006196402700A90000112063242B142B268
:1004D3001206196403700D900001120632FEF452E5
:1004E300B1EE42B2EF64047046120619FE700B902F
:1004F3000001120632F452B352B4EE6401700B9051
:10050300000112063242B3F452B4120619640270A7
:100513000A90000112063242B342B4120619640370
:10052300700D900001120632FEF452B3EE42B4EFA6
:1005330064057046120619FE700B90000112063214
:10054300F452C952CAEE6401700B900001120632D4
:1005530042C9F452CA1206196402700A90000112C9
:10056300063242C942CA1206196403700D90000193
:10057300120632FEF452C9EE42CAEF640670461206
:100583000619FE700B900001120632F452CB52CCC6
:10059300EE6401700B90000112063242CBF452CC90
:1005A3001206196402700A90000112063242CB420D
:1005B300CC1206196403700D900001120632FEF48A
:1005C30052CBEE42CCEF64077049120619FF7E004E
:1005D300700B900001120632F452E152E2EF640113
:1005E3004E700B90000112063242E1F452E2120601
:1005F300196402700A90000112063242E142E212CB
:1006030006196403700D900001120632FFF452E1E3
:10061300EF42E27F0022BB010689828A83E02250F7
:1006230002E722BBFE02E32289828A83E49322BB90
:10063300010CE58229F582E5833AF583E022500631
:10064300E92582F8E622BBFE06E92582F8E222E5E7
:100653008229F582E5833AF583E4932275F00875E0
:100663008200EF2FFFEE33FECD33CDCC33CCC582EA
:1006730033C5829BED9AEC99E58298400CF582EEA6
:100683009BFEED9AFDEC99FC0FD5F0D6E4CEFBE48E
:10069300CDFAE4CCF9A88222B800C1B90059BA0056
:1006A3002DEC8BF084CFCECDFCE5F0CBF97818EFB1
:1006B3002FFFEE33FEED33FDEC33FCEB33FB10D7B2
:1006C30003994004EB99FB0FD8E5E4F9FA22781873
:1006D300EF2FFFEE33FEED33FDEC33FCC933C910CE
:1006E300D7059BE99A4007EC9BFCE99AF90FD8E000
:1006F300E4C9FAE4CCFB2275F010EF2FFFEE33FED2
:10070300ED33FDCC33CCC833C810D7079BEC9AE844
:1007130099400AED9BFDEC9AFCE899F80FD5F0DAC5
:10072300E4CDFBE4CCFAE4C8F922EB9FF5F0EA9EB2
:1007330042F0E99D42F0E89C45F022E8600FECC3EB
:1007430013FCED13FDEE13FEEF13FFD8F122BB01F3
:100753000DE58229F582E5833AF5830207A0500768
:10076300E92582F8020793BBFE07E92582F8020711
:10077300ACE58229F582E5833AF5830207B9BB012B
:100783000689828A83F0225002F722BBFE01F322FC
:10079300E6FB08E6F908E6FA08E6CBF822E0F8A358
:1007A300E0F9A3E0FAA3E0FB22E2FB08E2F908E2A6
:1007B300FA08E2CBF822E493F8740193F9740293F4
:1007C300FA740393FB22FAE6FB0808E6F925F0F630
:1007D30018E6CA3AF622D083D082F8E493701274F2
:1007E3000193700DA3A393F8740193F5828883E4B6
:1007F300737402936860EFA3A3A380DF8B128A1341
:100803008914EF640260030208FA752202F523F5E6
:1008130024F525F526F527F528FFEFC3948074808A
:100823009480500F74802FF582E43400F583E4F054
:100833000F80E7E4FFEFC3948074809480500F74BB
:10084300002FF582E43400F583E4F00F80E7AB1268
:10085300AA13A914120619FF7E0064C06005EF6491
:10086300407077EF64C04E7005439A808003539ABB
:100873007F9000021207517F007E607D547C00123E
:10088300069B8F188E178D168C15E4FFFE7D01FCD9
:10089300AB18AA17A916A815C312072D40037FFF8B
:1008A30022C3E49518F518E49517F5177401951606
:1008B300F516E49515F515538EEF538EF7438E0415
:1008C300AF18AE17AD16AC15780812073E8FD68554
:1008D30018D753AFFB438E1080037FFF22AB12AABE
:1008E30013A914900007120632C454F0FFE59A547A
:1008F300EF4FF59A7F00227FFF221209F3120003C4
:10090300D2AF7BFF7A0A791E1200A87F017E001204
:100913000028D3E52794007480948040EE1527E5E2
:100923002770E8D3E526940074809480401EE4F594
:1009330008E508C39526501474002508F582E434AD
:1009430000F583E0FF120A0F050880E5E4F5268031
:10095300BAC0E0C083C082C0D075D000C007E59A9A
:1009630030E029539AFEE5287022C3E5269480746B
:100973008094804003752600AF26052674002FF56A
:1009830082E43400F583E59BF0752705E59A30E1B1
:1009930006539AFD752500D007D0D0D082D083D0DE
:1009A300E032EFD39401748094805007E5AF54FE96
:1009B3004FF5AFEDFF7E00D3940374809480502DE8
:1009C300EF700653B6FE53B5FEEF64014E70065347
:1009D300B6FE43B501EF64024E700643B60153B54C
:1009E300FEEF64034E700643B60143B5017F002258
:1009F300750A03E4F509FB7A0079097F010203A272
:100A0300787FE4F6D8FD7581280208FD8F9B752554
:100A130001E52570FC22AE07020A0F535443382028
:100A2300554152543220546573742050726F67726B
:080A3300616D6D65210D0A00E3
:00000001FF
